:10000000AA286D301A22851DCE280108850C0319F7
:100010000328800C850C800C850C800C850C800CD2
:10002000850C800C850C800C940A850C800C850C4A
:10003000800C840A850C800C850C800C1408850CBF
:10004000800C850C800CC039850C800C850C800CD4
:10005000CD3E850C800C850C800C840A850C800CB0
:10006000850C800C850C82009834963480340F34D3
:100070004234403401348634A03400342734103400
:1000800000340334E8340034003464340034003481
:100090000A34D334C034C434CB34532A003401344A
:1000A000043405341034113414341534D334C034CA
:1000B000CD34CF34D134D334C834CD34CF34D1342B
:1000C000043408341034203405340A341434283409
:1000D000BC345E342E3417340B340534033401340D
:1000E0004D3448347A34AF344F3466346634203477
:1000F000443469347334633468342E3420344334E4
:100100006834613472346734E53441346E346134B8
:100110006C3479347A346534F2345334653472345F
:1001200069346134EC344634723465347134753476
:1001300065346E346334F93456346F346C3474344B
:100140006D34653474347234F93442347234653445
:100150006134EB348316860183120C308600AC23A5
:1001600086100230E9232830CF230630CF230D300C
:10017000CF234030CF234E308F0020309600053003
:100180009400A923D923940BC1281530D623D72353
:100190008F0A960BBF2884308A23CF28DB23602266
:1001A000563045210318D6283F21D028110BE128CD
:1001B000950A1512B822150A6E23CF2810308C0626
:1001C000CF281118FC299118DE281119A9298C3083
:1001D0008A23EF280408263A031D942ADB23C8301B
:1001E000CF238C109F011D0A8E0073308E190729B2
:1001F0008C149F1440308E0A8E1907299F010330FA
:100200009E0003109E0D9F0D8E0B01291E0870236A
:10021000D723CC30CF2320300D196930D823373085
:100220008D1C3830D82320300D187030D823882208
:100230005B30452103181E293F21EF2811198F2A11
:10024000911C27291118FB2A8D0A8D11EF28111CEA
:10025000C42A9D0A9D11EF28B123DB2331298B236A
:10026000372BB82211183E2986100301F123ED2304
:100270002030F1230614851D2C29B1239129910AE0
:100280001119111C0800910108001107AA23CF239E
:100290009C01121413140E08F0388F008F0F4E2992
:1002A000010803195529901581012830051A3830A5
:1002B0008316810083121910181004308606051A5F
:1002C0006529061D18140C116829061919140C1536
:1002D0008C139808031D8C17980D0C139908031D97
:1002E0000C17990DF0238E0F4B298C1290080319CF
:1002F0007E29900318081904031D8C16050E8F0023
:100300008F098F0D930D03101303031908008F0D30
:10031000920D03141203031908009B0B4B299C0B2D
:100320004B299421860193299C010519851D942947
:10033000D0239C0B95290800D7235E30D8231B08B7
:100340006E2B9C2135309B0AA7219C214F309B0AA4
:10035000D82BCE230310170D9B009B0D9B07A121CB
:10036000A12194216022970A1719171CB829970117
:100370001708031DDC21C022143096008F01D02104
:100380008F0DD0218F0DD0210F0DD923960BBE29B3
:100390001708043C031DDC21CE21CF28CF21D0211A
:1003A0004B30840026309400031026180314800C70
:1003B0008403940BD72908008F008F0E8F028F03C0
:1003C0008F038F03CE218F0BE229080026301A22DB
:1003D000851DCE2801080319E8298403850C840AA9
:1003E000800C06308E00850C800C8E0BF329850C5A
:1003F000800C940BEE29532AB82215080319012802
:100400008F008F0B032A8F0B282A1722851DCE28D9
:1004100001080319062A0C2A850C800C14030739DD
:100420000319840A940B0B2A9C0B0C2A532A0230C2
:100430009C003030940026308400283006110C1ABD
:10044000232A3830061583168100831281010800A3
:100450000F03303E55228F001722851DCE2801083C
:1004600003192D2A8616850C800C140307390319ED
:10047000840A9519151D4B2A0F08960052308E00DC
:10048000D3230000960B3E2A0608DF39141E2038BD
:1004900086004E304D2A4C2A0F088E00D223940B32
:1004A000332A9C0B332A9701B829890003399F000E
:1004B0008316081483120808890A9E008C1008000D
:1004C000CE230D30960015081507150755229B0001
:1004D0001B0E56221B1B8C1471234D309508031DD7
:1004E0004B309B1BD8237030DD231B0856221B1971
:1004F0008C147123E4309B1D6D30D8237330D823C6
:100500002030D923960B802A01300C1E0430D623CC
:100510002A30D623170AC923D7237E30D82B970A2F
:100520001719971C942A9701253017191C3E971804
:100530000E3E1718073E8400C02207308F00840A41
:10054000000EF8230008F823D7238F0B9F2A0408F6
:10055000F93E8400CE2307308F00840A00087F39DB
:10056000E03E203E0318A530D8238F0BAD2AEF289C
:1005700014309700C022D723970BBB2A1F308C055D
:100580008030CF2B9A0A1A1162239421D330CF23C3
:100590009F01A001A1018F01F53096002530970041
:1005A0001A08203E2322851DC22A01089E001E0D26
:1005B0008F0D0F080339023A031DDF2A9F0A031922
:1005C000A00A9B30051D2F29970BD32A960BD52AFD
:1005D0001A0A9600960A03109E0D9F0DA00DA10DFC
:1005E000960BEB2A8830CF238F239B0BC62A1B1533
:1005F0009C0BC62A912906110D190615AB232F3025
:10060000B922263084001D08683EAA238E0094017A
:1006100094150D1C8D1C940A0D188D1894030D1D36
:10062000182B051E112B851DEA28051A132B1E2BCE
:10063000051A182B851DEA28051E1A2B86160000A0
:100640008E0B1E2B8E00A3238E0B232BA523850C34
:10065000800C940B222B0D18800D0D1D80090310AA
:100660008D18800C840A041B041E062B942A831602
:1006700085118312073096009E01851186155D2332
:1006800085181E1486119E0D960B3E2B8615851817
:100690001E1485151E0D8F0D0F080339023A031D18
:1006A000522B9F0A0319A00A9B30051D2F29883061
:1006B000CF238F23051DAA28372BFF30A800A80BB6
:1006C0005F2B080092308B23CE2364306C236F3075
:1006D000DD235230D82360301A07AA238C109F01E3
:1006E0009E00A101A001A501A401A3016430812302
:1006F000031DC9230A308123C9232E308C18D82327
:100700009E2BA2009401940AA0230318832BB423E8
:100710001403080097018F003B30B922DE2B3330E1
:100720008F008C11A501A823A400A823A300A8234F
:100730008123C3230F08B93E031C922B1E08C92B2B
:10074000A223B423A209A309A409A509A20A0800A7
:100750008F0A0F088200263084008001840A841FDB
:10076000AD2B940BB12B080022089E072308031819
:10077000230F9F0724080318240FA0072508031838
:10078000250FA10708008C19C92B003E0319D72B90
:100790008C150F3903191F30303ED82BC030E5239C
:1007A0008E010E17D32B8E0BD22B0800D8232030AE
:1007B00096038614E62BC022A4308F00A823803E27
:1007C0000318D82B7F39D823DE2B86108E00F12317
:1007D000ED230E0EF123ED23D02B0614EF2B061084
:1007E0000C080612861206138613F03986040800D8
:0E07F0000F399E00F63E031C9E2B413ED82B77
:02400E00F23F7F
:104200008800010001009800F40002008C00E40026
:104210002C00880064000A00880032001400D800D6
:1042200080001A00880019002800C800C00034006F
:1042300088000A006400C80060006800C800300000
:10424000D000C9001800A100800001000100140086
:1042500090001900000064000A0000002800190006
:10426000010006000900100016002E003000640056
:0A427000CC0005000E003B00950095
:00000001FF
